:020000040000FA
:020000002228B4
:08000800FE00030E8301C60097
:100010000A08C7008A0119280830C8000310C20D59
:100020000310C00D031C16284108C207C80B0E2878
:1000300008004808C9004008C3004108C40042083D
:10004000C5000129831605108510051105124F29D9
:1000500003108312500CE5004F0CE4000310E50C74
:10006000E40C64084F06E60065085006E70003103C
:10007000500CE9004F0CE8000310E90CE80C0310E9
:10008000E90CE80C68086606EA0069086706EB00F8
:100090000310500CED004F0CEC000430C0000310B6
:1000A000ED0CEC0CC00B4F286C086A06EE006D08D6
:1000B0006B06EF0001306E05E200E3010310500C07
:1000C000E5004F0CE400E601E7016218E717660857
:1000D0006404CF0067086504D0004F08C0005008D2
:1000E000C100080012150800831212117D147D084A
:1000F0008500FD147D0885007D157D0885000800BC
:100100007420282083124008DB0028208312400836
:10011000DC00282083124008DC0087309205FC3088
:100120009205C330831692008312D70183168C1474
:1001300083128C1072284A108C1CA32883168C1CE6
:10014000A32883124A1483124A1CE7288C107D16B8
:100150007D0885005708031DBF283330D7005B0892
:10016000D8005C08D9005D08DA007D107D088500A4
:10017000FD107D0885007D117D088500C028D7030E
:10018000053058020319C628031CC9280530D802B7
:10019000CC287D147D088500053059020319D2282A
:1001A000031CD5280530D902D828FD147D08850008
:1001B00005305A020319DE28031CE1280530DA0253
:1001C000E4287D157D0885007D127D0885004308A3
:1001D000C0004408C1004508C2004908C8004708DB
:1001E0008A00460E8300FE0E7E0E09001030831634
:1001F0009F00953083129F0060100C1383160C171C
:1002000008004E100C1F092983160C1F09298312A0
:100210004E1483124E1C9B28601825291E08C0000E
:10022000FF30C1000C2083124208CA00CB018316A4
:100230001E088312CC00CD014D084B07D2004C089C
:100240004A07D1000318D20A60140C139B288312AA
:10025000601C31295108D3005208D40060104014AA
:100260000800401008009F140800803083129F008F
:10027000080074203521BA308312D600831203138C
:100280009C30C0007F30C1000A128A11C10B442982
:100290000A128A11C00B4229000063000800831271
:1002A00003139C30C0007F30C1000A128A11C10BB9
:1002B00055290A128A11C00B532900007420BA3044
:1002C00083125602031D6729D630D60068293921CA
:1002D00083124F085004031D7129E130CF00AC3068
:1002E000D000F62080208312D5010B178B173F30EA
:1002F00083169500811327218312E0114018E01521
:10030000E01D962900305402031D8829C83053028D
:1003100003199529031C95290A305502031D9329B9
:10032000D50139219629D50A9629D501282083128D
:100330004008DE004108DF001F305F02031DA229D4
:10034000FF305E020319AF29031CAF29FA305B02AC
:100350000319B7290318B7290530DB07B729463039
:100360005B020319B729031CB7293230DB022820AE
:1003700083124008DE004108DF001F305F02031DCA
:10038000C329FF305E020319D029031CD029FA309B
:100390005C020319D8290318D8290530DC07D829AD
:1003A00046305C020319D829031CD8293230DC02FC
:1003B000282083124008DE004108DF001F305F0262
:1003C000031DE429FF305E020319F129031CF12902
:1003D000FA305D020319F9290318F9290530DD0700
:1003E000F92946305D020319F929031CF929323035
:1003F000DD023321831203139330C0001A30C10091
:100400000A128A11C10B002A0A128A11C00BFE2996
:0C041000000000000000000000007B293C
:02400E00643C10
:00000001FF
